:1000000001308A00A12900002E30840083130008EB
:10001000031917280230F800F701F70B0D28F80B29
:100020000C289730F700F70B1328800B0A280800DC
:100030000511051707128712071707118710851773
:100040008715851105158A110A12712A8F018E01F3
:100050000130AE0004200F08FA000E08F7000F0868
:100060007A02031D2B287708AC007A08AD002D0812
:10007000083C031C4328031D41282C08973C031C03
:1000800043288A010028080085178715B60136081D
:10009000073C031C5628B41F4F280715502807118A
:1000A000871487100310B40DB60A4728B601360826
:1000B000073C031C6628B51F5F2807156028071139
:1000C000871487100310B50DB60A572808003208A8
:1000D000B4003308B50044208513851708003208A2
:1000E000B4003308B50044208711871508000511B6
:1000F000051307128716071707118710851787152D
:10010000851105150130AE00042026201230B20002
:100110008030B30067201430B2008030B3006F200D
:100120008A110A12712A051105130716871207177B
:100130000711871085178715851105150130AE0049
:10014000042026201230B2008030B3006720143023
:10015000B2008030B3006F208A110A12712A051193
:1001600005130712871207130711871085178715C4
:10017000851105150130AE00042026201230B20092
:10018000B30167201430B200B3016F208A110A1244
:10019000712A051105130716871607130711871013
:1001A00085178715851105150130AE00042026201E
:1001B0001230B200B30167201430B200B3016F20D7
:1001C0008A110A12712AB301B201B40134080F3C3A
:1001D000031C0C299F1435109F1C35143518F42866
:1001E00035109F1C3514EE289F18F4281E08FA00BD
:1001F00083161E088312B6001E08B7003608F800E2
:100200003708F9007908FA007808B2077908031866
:10021000790FB307B40AE628B30CB20CB30CB20CD6
:10022000B30CB20CB30CB20C0F30B305220B462941
:1002300021083302031C2A29031D22293208200227
:1002400003182A293308A1003208A000F800210869
:10025000F900782901303207F8003308FA00031852
:10026000FA0A7A082102031C4529031D3B292008AC
:100270007802031845293308A1003208A000A20122
:100280002008F8002108F900782974293308210290
:10029000031C5829031D502920083202031858292D
:1002A0003308A1003208A000F8002108F9007829DD
:1002B00001302007B5002108B6000318B60A360839
:1002C0003302031C7429031D6929320835020318FF
:1002D00074293308A1003208A0000130A2002008D0
:1002E000F8002108F90078292008F8002108F90011
:1002F0007908AD007808AC0023082C02031D84297E
:1003000024082D0203199E292D08A4002C08A300FF
:100310002C08AF00B3012D080339AE002E080438B5
:10032000B0002E080C38B1003008B2002F08B3001E
:1003300067203108B2002F08B3006F208A110A121B
:10034000732A840183131F308305713083168F0055
:100350000F088312A101A0010130A2000330A40004
:10036000FF30A300FF30A500831603170908C0392A
:10037000890003131F129F12003003178800831295
:10038000870188018901FF308316031395008113CB
:100390008500860087008612831286128316061354
:1003A0008312061383168613831286130230AC0061
:1003B000FA30AE000420AC0BD829073090001F1390
:1003C0009F1783169F1783121F148316031709089C
:1003D000C039890003131F129F12013003178800D0
:1003E0000030F800831203131F08C33978049F00FC
:1003F000A51325088316870085100511051285129F
:100400000511831205118316851183128511831638
:10041000851383128517A51125088316870083127B
:100420008715A510250883168700831287142511C8
:100430002508831687008312071583160513831278
:100440000517251225088316870083120712A512A7
:100450002508831687008312871225132508831623
:1004600087008312071705150130AE000420053000
:10047000A600AB01AA012B08A9002A08A800A70121
:100480000618442A0130A7008618482A0230A7001F
:1004900006194C2A0330A7008619502A0430A700F9
:1004A000270826020319712A2708A600260803191F
:1004B000662A013A0319682A033A03196A2A013A9B
:1004C00003196C2A073A03196E2A702A1828712A10
:1004D0007728712A9328712AAF28712AC928712A8E
:1004E000712A8616E32886122908023C0318812AFD
:1004F000FF3A031D7F2A2808E83C0318812A0617C3
:10050000842AA80A0319A90A2B08083C0318912A6F
:10051000FF3A031D8F2A2A08C43C0318912A861724
:0C052000942AAA0A0319AB0A3F2A6300C0
:04400E00842CFF3FC0
:00000001FF
